:100000000C94D9010C9411020C9411020C9411025D
:100010000C9411020C9411020C9411020C94110214
:100020000C9411020C9411020C9452220C9424236F
:100030000C94311D0C9411020C9411020C941102B9
:100040000C9411020C9411020C9411020C941102E4
:100050000C94A1170C94B91D0C9411020C9411026C
:100060000C9411020C9411020C9411020C941102C4
:100070000C9411020C9411020C9411020C941102B4
:100080000C9411020C9411020C9411020C941102A4
:100090000C9411020C9411020C9411020C94110294
:1000A0000C9411020C9411020C9411023F053F05AF
:1000B0006B056B05D305F10509070907FC059506D6
:1000C000A606A606B016B216B716BA16BD16C01604
:1000D000C3169123B823B024B823B02404242724C2
:1000E000B0247E248D24AC00A800AB00AD00AE008F
:1000F000AF00B200B100B341C05C0100C25CBF5CA4
:10010000BE5CC15CBC5CBD5C010000000000000086
:1001100000002A2B28000000000000000000000062
:10012000000000000029000000002C1E34202122C5
:1001300024342627252E362D3738271E1F2021222E
:10014000232425263333362E37381F0405060708A7
:10015000090A0B0C0D0E0F10111213141516171897
:10016000191A1B1C1D2F3130232D350405060708D5
:10017000090A0B0C0D0E0F10111213141516171877
:10018000191A1B1C1D2F3130354C000000000000D7
:10019000000000000000000000000000000000005F
:1001A00000000000000000000000000000007E0FC2
:1001B00000D4FFFFFFC7000000780000000000002F
:1001C000000000000001010203040506080A0C0FEC
:1001D0001114181C2024292E33393F464C535B62DE
:1001E0006A7179818A929AA2AAB2B9C1C8CFD5DCC4
:1001F000E1E7EBF0F4F7FAFCFDFEFFFEFDFCFAF799
:10020000F4F0EBE7E1DCD5CFC8C1B9B2AAA29A926B
:100210008A8179716A625B534C463F39332E2924B7
:10022000201C1814110F0C0A080605040302010112
:100230000000000000000000000014034E00430016
:10024000430031003700300031004B004200000015
:1002500018034A0032004C0020004400650073007F
:10026000690067006E0073000000040309040902BE
:100270003B00020100A0FA09040000010301010093
:100280000921110100012240000705810308000136
:1002900009040100010300000009211101000122ED
:1002A000B6000705820320000112010002000000D1
:1002B00008EDFE011701000102000105010902A17C
:1002C0000185020901A10005091901290815002568
:1002D0000195087501810205010930093115812553
:1002E0007F95027508810609381581257F9501756E
:1002F000088106050C0A38021581257F95017508CD
:100300008106C0C005010980A101850319012AB732
:1003100000150126B700950175108100C0050C0974
:1003200001A101850419012AA002150126A0029548
:100330000175108100C005010906A10185060507A8
:1003400019E029E7150025019508750181020507C7
:10035000190029EF1500250195F0750181020508A6
:100360001901290595057501910295017503910102
:10037000C005010906A101050719E029E7150025B7
:10038000019508750181029501750881010507191C
:100390000029FF150026FF00950675088100050855
:1003A00019012905950575019102950175039101C2
:1003B000C00011241FBECFEFDAE0DEBFCDBF04B610
:1003C00003FE18C080919E0290919F02A091A0020E
:1003D000B091A1028730904BA740B04B59F41092D6
:1003E0009E0210929F021092A0021092A102E0E0E1
:1003F000F8E3099511E0A0E0B1E0EEE5FBE402C00E
:1004000005900D92A439B107D9F722E0A4E9B1E033
:1004100001C01D92AE39B207E1F70E94F1120C94AF
:10042000AD250C940000823038F4662311F089EA7F
:1004300001C08AEA0E94ED0481E008959C013A958A
:1004400021153F4130F5BC0166277270AC0144278D
:1004500054709C012227387094FF0FC090FF02C097
:1004600080E101C080E0672B09F08062452B09F034
:100470008064232B79F080680895892F8170672B21
:1004800009F08260452B09F08460232B19F0886005
:10049000089580E00895CF93DF93EB010E941E0240
:1004A000FE01DF91CF910994CF93DF93EC01805E41
:1004B0009109089710F0209719F466EF74E002C0D4
:1004C00061E877E0CE010E944B028C2FDF91CF9143
:1004D0000C944C04CF93DF93EC010E94A204CE0154
:1004E000805E9109089710F0209719F46DEF74E081
:1004F00002C068E877E0CE01DF91CF910C944B0207
:10050000CF93DF93EC010E945402C933D10549F423
:100510002FEF87EE93E0215080409040E1F700C03C
:100520000000CE01DF91CF910C946A0281E0089522
:1005300081E008950C94980208950C949C021F93F6
:10054000CF93DF9300D000D01F92CDB7DEB74983A1
:100550005A836B833091970189819A81311114C03C
:10056000662359F0222349F00E945409182F682F5E
:1005700089819A810E94FD0803C00E942809182FD2
:1005800069817A81812F04C00E94540969817A812E
:100590000F900F900F900F900F90DF91CF911F91C0
:1005A0000C949410FC01262F40815181628173814B
:1005B00084810C949F0281E00895CF93DF93EC0136
:1005C00060E00E94D202BE01DF91CF910C949D02A7
:1005D0000C94C3110C94BF1108950E94A7070E94A8
:1005E000EC022FEF84E39CE0215080409040E1F743
:1005F00000C000000C94DF1D0F931F93CF93DF9377
:100600008C0161E00E94D202EC01B8010E949A02C2
:10061000882309F44BC0B801CE010E94A11688239B
:1006200009F444C0B801CE010E9409198823F1F1F0
:10063000B801CE010E947A1B8823C1F1B801CE0116
:100640000E942719882391F1B801CE010E94D61A81
:10065000882361F1F8018281882309F1CB358DE58A
:10066000D807C1F050F4C115FCE5DF0781F0CF3D9C
:10067000DC45A9F40E94880E19C0CC35EDE5DE07F3
:1006800061F0CD35DD4559F40E94D10D08C00E94BE
:10069000ED020CC00E94DA0D02C00E94DD0DC801FF
:1006A000DF91CF911F910F910C94960280E0DF9122
:1006B000CF911F910F9108950E94141D80E00E9418
:1006C00059170C94EA030E94C5150E94ED030C947F
:1006D0001A1DDF92EF92FF920F931F93CF93DF9338
:1006E000E82FF0E0E65FFE4FD490282F2695269560
:1006F000269530E0F901E655FE4F0491877010E031
:10070000082E02C0159507950A94E2F7017011278B
:10071000F901E656FE4FE490F12C082E02C0F59444
:10072000E7940A94E2F791E0E922FF24F901E65701
:10073000FE4FC491D0E002C0D595C7958A95E2F7E7
:10074000C170DD270115110519F081EE0E944C04DE
:10075000E114F10419F086EE0E944C048D2D0E94E4
:10076000ED04EF2819F086EE0E94A204012B19F087
:1007700081EE0E94A204CD2B51F08CE2DF91CF914B
:100780001F910F91FF90EF90DF900C94ED04DF919B
:10079000CF911F910F91FF90EF90DF900895982FC8
:1007A0009F709A50963010F0805D01C0895A0C9469
:1007B000690308950C94D90381E008950C94DC0337
:1007C0000895CF93C82F0E94DA038C2F0E94DE0376
:1007D000CF91089580E00C94E1030E94D61B0C9405
:1007E000E1030E94D61B90919601891721F0809316
:1007F00096010C94E1030895CF93DF93CDB7DEB754
:100800002B970FB6F894DEBF0FBECDBF4F8358872E
:1008100069877A878B8761110E941D0D9E012F5F6A
:100820003F4F86E0F90111928A95E9F785E0FE01D4
:100830003796D90101900D928A95E1F789819A81C5
:100840004C815D81452B31F09F3F31F491E08F3F2A
:1008500019F403C091E001C090E090FF09C0498104
:100860005A816B817C818D819E810E943B0C05C0E9
:10087000C9010E94DB028111F2CF2B960FB6F894CA
:10088000DEBF0FBECDBFDF91CF910895FC01808107
:1008900091810E9496090895CF93882309F450C04E
:1008A000C82F8CEF8C0F813AD0F46C2F809102010D
:1008B000909103010E944F1C882349F06C2F809176
:1008C0000201909103010E94DA1C0E943F0D6C2FDF
:1008D00080910201909103010E94CF1C0CC080E224
:1008E0008C0F883058F4C77081E001C0880FCA951A
:1008F000EAF70E94FD0CCF910C943F0DEBE5EC0F55
:10090000E33040F4F0E0E75BFE4F808190E0CF9170
:100910000C940D1CE8E5EC0FE73150F4F0E0EE0F1D
:10092000FF1FE55EFE4F80819181CF910C94231CC7
:10093000CD3E30F08C2F0E947613CF910C9448144A
:10094000CF910895882389F19CEF980F913A40F454
:10095000682F80910201909103010E94DA1C0DC062
:1009600090E2980F983058F4877091E001C0990F89
:100970008A95EAF7892F0E94030D0C943F0D9BE5A1
:10098000980F933020F480E090E00C940D1C98E5D3
:10099000980F973120F480E090E00C94231C8D3E5A
:1009A00020F00E94D1130C94481408951F93CF9304
:1009B000DF93182FEB010E944C04209741F08FE940
:1009C0009FE00197F1F700C000002197F6CF812F3B
:1009D000DF91CF911F910C94A204893319F060E04C
:1009E00070E002C060E570E00C94D604882321F02A
:1009F0000E94FD0C0C943F0D0895882321F00E9465
:100A0000030D0C943F0D0895CF92DF92EF92FF9269
:100A10000F931F93CF93DF937C01D62FC72FFC0139
:100A20001281058102950F700E94F30C8823B9F0A2
:100A30001123A9F08C2F807F803421F080E28D0F6C
:100A4000883068F080917E0282FD09C082E00E94B9
:100A50009F0D0E94F30C91E0D82ED92601C0D12C15
:100A6000CC2EC2948FE0C8228C2D90E08C30910562
:100A700008F0CFC1FC01EA5AFF4F0C943E258C2FA1
:100A8000807FCF70882311F0C295C07F112399F029
:100A9000CC2309F4AAC180E28D0F883010F0D11167
:100AA00004C08C2F0E94FD0C03C08C2F0E94100DDF
:100AB0000E943F0D9AC18D2F0E94A204CC2309F4FD
:100AC000A8C180E28D0F883038F1DD2329F18C2F09
:100AD0000E94160D24C08C2F807FCF70803211F0C1
:100AE000C295C07FDD2319F0D130A1F13DC08091C6
:100AF0007E0282FF17C0112349F0CC2329F08C2FEE
:100B00000E94FD0C0E943F0D80E070C180E00E94B9
:100B1000A204CC2309F47DC18C2F0E94030D0E94F6
:100B20003F0D77C1112371F0002341F0013031F402
:100B30000E94200D8C2B0E94280D6BC10E94200D5D
:100B40008C2B1DC0002319F0013009F462C10E94F2
:100B5000350D25C0112321F0063008F05AC10EC012
:100B6000053008F056C11BC0112361F0002331F09D
:100B7000F701858180FF39C18F7085838C2F0E949A
:100B8000F60447C1002359F0D93309F03FC1FFEF04
:100B900007EE13E0F15000401040E1F735C18C2F13
:100BA0000E94FD0436C18C2F86958695837019F0BE
:100BB000813061F02EC1112321F08D2F9C2F937075
:100BC00002C080E090E00E940D1C2BC1112321F097
:100BD0008D2F9C2F937002C080E090E00E94231C18
:100BE00020C18D2F112319F00E94761302C00E949C
:100BF000D1130E94481415C18C2F837009F047C08F
:100C000011110BC12D2F229526952770220F220F2F
:100C10006D2F6F70862F90E0A0E0B0E0022E04C030
:100C2000880F991FAA1FBB1F0A94D2F7D4FF10C0C8
:100C30004FE050E060E070E004C0440F551F661FB5
:100C4000771F2A95D2F7409550956095709503C00F
:100C500040E050E0BA01C695C695C3708A019B0179
:100C6000082B192B2A2B3B2BC901B801C23049F0A4
:100C700058F4C13019F00E941308CFC00E94010837
:100C8000CCC00E942508C9C00E94FF07C6C011231E
:100C900019F08C2F817001C08695882309F4BDC09E
:100CA0002D2F229526952770220F220F6D2F6F7002
:100CB000862F90E0A0E0B0E0022E04C0880F991FBC
:100CC000AA1FBB1F0A94D2F7D4FF10C04FE050E018
:100CD00060E070E004C0440F551F661F771F2A951F
:100CE000D2F7409550956095709503C040E050E074
:100CF000BA01C695C695C3708A019B01082B192BB2
:100D00002A2B3B2BC901B801C23049F058F4C1303D
:100D100019F00E94D80881C00E94C6087EC00E94B7
:100D2000EA087BC00E94390878C0CF70112339F0DF
:100D30008C2F0E945F088D2F0E94F6046EC08D2FAD
:100D40000E94FD048C2F0E94800867C0D23F21F1D1
:100D500028F4D03F41F0D13FC1F043C0D33F19F157
:100D6000D43F79F03EC0112341F0053008F051C066
:100D70008C2F8F710E94A5084CC0063008F049C026
:100D8000F7CF80917E0282FF18C0112339F08C2F9B
:100D90008F710E945F083DC01123C9F38C2F8F71A2
:100DA0000E94800836C0112329F08C2F8F710E9479
:100DB0004A082FC00E9445082CC0112349F0CF716A
:100DC0008C2F0E945F0863E08C2F0E94840D21C04D
:100DD00081E00E949F0D0230E0F082E00E949F0DB2
:100DE00018C0112331F0002391F28D2F0E944C0482
:100DF00010C0002399F2D93349F41FEF27EE33E0F6
:100E0000115020403040E1F700C000008D2F0E94BB
:100E1000A20488EF8C0D843020F40E94D61B0E941F
:100E2000E103DD20C9F00E94EF0C80FD15C0F70141
:100E300012820E94E90C0E945F08C7010E944D07C0
:100E40000E94E90CDF91CF911F910F91FF90EF90DD
:100E5000DF90CF900C948008DF91CF911F910F917C
:100E6000FF90EF90DF90CF9008950F931F93CF9353
:100E7000DF93EC01688179818A810E94A1098C014C
:100E80000E94FC080E94ED07B801CE010E940405F3
:100E9000DF91CF911F910F910895CF93DF93EC01D4
:100EA000988189812B813C81232B31F08F3F31F454
:100EB00081E09F3F19F403C081E001C080E080FD24
:100EC0001DC0CE010E94FC02811110C00E94F30CD3
:100ED0008823A1F08A81882389F080917E0282FD97
:100EE0000DC082E0DF91CF910C949F0DCE010E9446
:100EF0003507CE01DF91CF910C94DD02DF91CF91C8
:100F00000895882321F00E94100D0C943F0D089540
:100F1000882321F00E94160D0C943F0D089580E067
:100F200090E00E940D1C80E090E00E94231C0E9433
:100F30001D0D0E943F0D0E9479150C94481480915C
:100F40000201909103010E94E51C0C948F070E94FE
:100F50000D0D0C949F0792959F70963079F010F4C8
:100F6000925001C09A50923068F4803F69F018F4B2
:100F7000883E40F409C0843F29F406C0883E20F032
:100F8000813F11F080E0089581E00895FC018081A7
:100F900091810E9496090E94AB070895CF93DF9339
:100FA00000D000D01F92CDB7DEB70F900F900F90FA
:100FB0000F900F90DF91CF910895CF93DF9300D0E2
:100FC00000D000D0CDB7DEB726960FB6F894DEBFBE
:100FD0000FBECDBFDF91CF910895089508950C9471
:100FE000EE070C94EF070E94F1076093A60170933F
:100FF000A7018093A8019093A9010C948F070C94EA
:10100000F3070F931F930091A6011091A701209160
:10101000A8013091A901602B712B822B932B1F917A
:101020000F910C94F3070F931F930091A601109159
:10103000A7012091A8013091A90160237123822387
:1010400093231F910F910C94F3070F931F9300911B
:10105000A6011091A7012091A8013091A901602754
:101060007127822793271F910F910C94F3070C94FB
:10107000EE070E9437086093A2017093A30180934A
:10108000A4019093A5010C948F0760E070E0CB0160
:101090000C9439080F931F9341E050E060E070E03A
:1010A0008A019B0104C0000F111F221F331F8A9564
:1010B000D2F7C901B8011F910F910C9439080F9311
:1010C0001F9341E050E060E070E004C0440F551F02
:1010D000661F771F8A95D2F78091A2019091A30194
:1010E000A091A401B091A5018A019B01082B192BA5
:1010F0002A2B3B2BC901B8011F910F910C94390881
:101100000F931F9341E050E060E070E004C0440F93
:10111000551F661F771F8A95D2F7409550956095A9
:1011200070958091A2019091A301A091A401B0912A
:10113000A5018A019B01082319232A233B23C90106
:10114000B8011F910F910C9439080F931F9341E040
:1011500050E060E070E004C0440F551F661F771F29
:101160008A95D2F78091A2019091A301A091A40148
:10117000B091A5018A019B01082719272A273B273F
:10118000C901B8011F910F910C9439080F931F9357
:101190000091A2011091A3012091A4013091A50119
:1011A000602B712B822B932B1F910F910C9439087C
:1011B0000F931F930091A2011091A3012091A4010C
:1011C0003091A50160237123822393231F910F91F6
:1011D0000C9439080F931F930091A2011091A30161
:1011E0002091A4013091A5016027712782279327C0
:1011F0001F910F910C9439080895292F220F920FF7
:10120000890FE82FE695E695E695877051E001C0D5
:10121000550F8A95EAF785E0E89FF0011124E8561A
:10122000FE4F20E030E070E04081CB01022E02C092
:10123000969587950A94E2F7817081958427852396
:10124000842781932F5F3F4F2530310569F708953B
:10125000292F220F920F890F682F66956695669544
:10126000982F977085E0689FB001112440E050E00E
:1012700080E0FB01E40FF51FE856FE4F208130E0CF
:10128000092E02C0369527950A94E2F7217033277C
:10129000042E01C0220F0A94EAF7822B4F5F5F4FA2
:1012A0004530510531F70895BF92CF92DF92EF920A
:1012B000FF920F931F93CF93DF938C01C090A201F5
:1012C000D090A301E090A401F090A5018091A60127
:1012D0009091A701A091A801B091A901C82AD92A8B
:1012E000EA2AFB2ACFE1D0E0D701C6010C2E04C0C8
:1012F000B695A795979587950A94D2F780FD04C077
:10130000219790F7B12C07C0BC2EB8018C2F0E94FA
:10131000AA100197A9F38B2DDF91CF911F910F9107
:10132000FF90EF90DF90CF90BF900895CF93DF9321
:10133000EC010E945409BE010E94AA10DF91CF91D6
:1013400008951F93CF93DF93EB0190919701992319
:1013500021F0CB010E94960913C0882349F0CB01EC
:101360000E945409182F682FCE010E94FD0804C066
:10137000CB010E942809182FBE01812F0E94AA10BC
:10138000DF91CF911F9108951F93CF93DF93C09169
:10139000AA0116E08091AB01C81799F0D0E01C9F1C
:1013A000F0011D9FF00D1124E455FE4F4081518145
:1013B00062817381848195810E94DD072196C770C7
:1013C000E9CFDF91CF911F9108954091DC015091B9
:1013D000DD016091DE017091DF018091E00190916B
:1013E000E1010C94DD07EF92FF920F931F93CF93CF
:1013F000DF938091E10182958F7009F065C0809143
:10140000DE01882309F460C08091AA01F090AB014D
:101410001091DC010091DD016091DF017091E0012C
:1014200091E01F3F09F090E0C0910001D0910101CF
:10143000292F96E0E92E8F1509F446C06115710534
:1014400021F00F3F21F030E003C031E001C0322F26
:1014500090E030FD36C0E89EF001E99EF00D1124C9
:10146000DF01A455BE4F11963C911197301329C04E
:101470003C91311326C012963C911297311121C034
:1014800013964D915C911497461B570B4C175D07B3
:10149000C0F48091E1018F7080618093E101EF548D
:1014A000FE4F80818F70806180838CED91E00E947F
:1014B0004D07DF91CF911F910F91FF90EF900C940A
:1014C000C40901968770B7CFDF91CF911F910F911B
:1014D000FF90EF9008959F92AF92BF92CF92DF92CC
:1014E000EF92FF920F931F93CF93DF93CDB7DEB7A9
:1014F00061970FB6F894DEBF0FBECDBF8C0185E0BB
:10150000F801DE011D9601900D928A95E1F7D80150
:101510001296EC909091DC01E091DD012091DF01C9
:101520003091E0012115310531F0EF3F31F481E0D8
:101530009F3F19F403C081E001C080E0B82FB17073
:101540009B2E80FD47C1D8014C9111965C9111975B
:101550001396AD90BC9014978CEDC82E81E0D82ED8
:10156000F090DE01B501621B730B209100013091F8
:101570000101FF2009F4D9C08091E10162177307CE
:1015800008F095C0282F207F09F052C05E1313C0C9
:10159000491311C0FE2CE1100EC08F708061809342
:1015A000E1010E94E509C6010E944D078091E10119
:1015B000F80185834DC1AB2831F05F3F31F481E004
:1015C0004F3F19F403C081E001C080E080FD03C0FB
:1015D00081E08E2502C080E090E0F82FF170FF2EB0
:1015E00080FF1CC08091AA012091AB0136E08217D8
:1015F00009F40BC190E0389FF001399FF00D1124E0
:10160000E455FE4F6181561306C06081461303C046
:101610006281E61203C001968770E9CFFE2CEE20AE
:1016200009F416C18091E10181608093E10154C009
:101630005E1306C0491304C0E11002C0F80199C04E
:10164000C8010E94C607882361F1EE2051F1209164
:10165000E101822F82958F7090E0029774F0809163
:10166000DC019091DD0198878F831986BB86AA865D
:101670002C87CE0107960E944D0786E0F801ACED5D
:10168000B1E001900D928A95E1F70E94F3090E9462
:10169000E5090AC05E1711F1C8010E94C607811151
:1016A0002CC0C8010E944D07FF24F394D1C0282FFD
:1016B000207F81F77A2DB98AA88A6E2D89890E94A8
:1016C000CE078CED91E00E944D0786E0D6011D9279
:1016D0008A95E9F70E94E509F12CBAC04913DCCFDD
:1016E000E110DACFF8018583C8010E944D0786E03A
:1016F000D6011D928A95E9F7ABC0EE2091F22091B8
:10170000E101822F82958F7090E002970CF4B5CFA3
:101710008091DC019091DD019A8389831B82BD82D7
:10172000AC822E83CE010196A6CF6217730708F014
:1017300044C0FE2CEE2009F4B4CF5E1330C0491330
:101740002EC02091E10120FD21C0822F82958F7053
:10175000482F50E041155105C9F0F80125834F305D
:10176000510541F08F5F982F9295907F822F8F7057
:10177000892B8583C8010E944D0786E0F801ACEDF6
:10178000B1E001900D928A95E1F73CC086E0F80146
:10179000ACEDB1E001900D928A95E1F759C0C80116
:1017A0000E94C607811169CF8091E1018160809319
:1017B000E101C8010E944D074BC07A2DB98AA88A61
:1017C0006E2D89890E94CE0786E0D6011D928A95EA
:1017D000E9F718C0EE2009F464CFC8010E94C607DB
:1017E000F82E882309F45DCF86E0F801ACEDB1E076
:1017F00001900D928A95E1F78CED91E00E944604EC
:101800000E94F3090E94E50923C04D875E878D85FC
:101810009E850E949609292F22952F70223028F448
:101820009F7039F0811105C00BC0243028F49F70DF
:1018300049F4805E883020F0C8010E944D079F2C3B
:10184000F92C06C0D80115969C91907F91F7F8CF9E
:101850008F2D61960FB6F894DEBF0FBECDBFDF911E
:10186000CF911F910F91FF90EF90DF90CF90BF909D
:10187000AF909F9008951F93CF93DF93CDB7DEB7BE
:101880002C970FB6F894DEBF0FBECDBF4F8358879D
:1018900069877A878B879C87CE0107960E946B0A9F
:1018A0008823D1F09F8188852A853B85232B31F0C1
:1018B0008F3F31F481E09F3F19F403C081E001C004
:1018C00080E080FD47C04F81588569857A858B858A
:1018D0009C850E94DD073EC086E0FE013796DE0152
:1018E000119601900D928A95E1F7FF81E8856A854E
:1018F0007B856115710531F0EF3F31F481E0FF3FE9
:1019000019F403C081E001C080E080FD23C0209174
:10191000AB0130E0C9010196877099274091AA0177
:1019200050E084179507F1F1F983EA837D836C8396
:1019300096E0929FD001939FB00D1124A455BE4F05
:10194000FE01319601900D929A95E1F78093AB01DB
:101950000E94C40916E08091AA019091AB018917F9
:1019600071F1189FC001112484559E4F0E946B0A8B
:10197000882329F1E091AA011E9FF0011124E4556A
:10198000FE4F4081518162817381848195810E94E3
:10199000DD078091AA0190E00196877099278093D6
:1019A000AA01D9CF0E94A7071092AB011092AA01F9
:1019B000ECEDF1E086E0DF011D928A95E9F72C96C7
:1019C0000FB6F894DEBF0FBECDBFDF91CF911F9150
:1019D0000895809102028595859585950895809159
:1019E00002028770089590910202977081E009F4D5
:1019F00080E0089580912502089590912502892B19
:101A000080932502089580959091250289238093E3
:101A100025020895809325020895109225020895C5
:101A200090912402892B80932402089580959091AF
:101A30002402892380932402089510922402089599
:101A400080910302089508950C94230D0C94240DA5
:101A500090917E0292FD08C090910302981721F0A8
:101A6000809303020C94260D08958091030288232D
:101A700029F01092030280E00C94260D0895CF9374
:101A8000DF93E0910201F0910301809125028083B0
:101A9000E0910201F0910301908180912402892B51
:101AA000808380910302882381F0E0910201F0910C
:101AB00003019081892B8083809102019091030121
:101AC0000E94391C81110E94350DC0910201D091F4
:101AD000030140E250E062EE71E0CE010E945E251B
:101AE000892B69F080E2FE01A2EEB1E001900D9237
:101AF0008A95E1F7CE01DF91CF910C94E51BDF9140
:101B0000CF9108950C94230D90917E0292FD10C008
:101B100098E0899F90011124262B209302020E94B5
:101B20005F08809102028595859585950C94820DBC
:101B30000C945F081092020280E00C94820D2091B8
:101B400002028095822380930202982F977099F465
:101B500030E0482F082E000C550B2417350759F09C
:101B600090917E0292FD07C08595859585950E948E
:101B700080080C949A0D089590917E0292FB222782
:101B800020F9281769F080FB92F990937E028091EA
:101B90007D0290917E020E94040E82E00C949F0DC3
:101BA000089580917E0282FB882780F991E0892741
:101BB0000C94BC0D81E00C94BC0D80E00C94BC0D29
:101BC00080E090E00E94732521E0893E9E4F09F05D
:101BD00020E0822F089582E090E00C946B2583E052
:101BE00090E00C946B25CF9384E090E00E946B25ED
:101BF000C82F82E290E00E946B252C2F30E0A901D3
:101C0000582BCA01CF910895CF93C92F682F84E034
:101C100090E00E9479256C2F82E290E0CF910C94A5
:101C20007925AB01BC018FE090E00C948B25AB01D2
:101C3000BC0183E190E00C948B2560E070E0CB0167
:101C40000C94170E60E070E0CB010E94110E0C9412
:101C50001D0E69EE7EEF80E090E00E94972560E027
:101C600082E090E00E94792560E083E090E00E94AD
:101C700079251092A6011092A7011092A801109246
:101C8000A90160E084E090E00E94792560E082E2B2
:101C900090E00E94792560E085E090E00E9479253F
:101CA00060E086E090E00E9479256FEF87E090E0A9
:101CB0000E94792540E050E0BA0188E090E00E945F
:101CC0008B2560E08DE090E00E94792540E050E0B7
:101CD000BA0188E190E00E948B2560E087E190E006
:101CE0000E94792540E050E0BA018CE190E00E942A
:101CF0008B2560E070E080E290E00E94972540E054
:101D000050E0BA0188E190E00E948B250C94220EED
:101D10000C94290E682F8EE090E00C9479250E9497
:101D20009E1D609331027093320280933302909330
:101D3000340260932D0270932E0280932F029093B1
:101D4000300208950E949E1D60933102709332020A
:101D500080933302909334026093290270932A0295
:101D600080932B0290932C02089585B7806885BFDD
:101D700085B7806885BF089581E008950C94BC0EF6
:101D800008950C94C00E0C94C00E0C94C30E0C94C9
:101D9000C00E0C94C70E0C94C00E0E94B50E86E8BF
:101DA00091E10E94CC1B0E94CB0E0C94C90E0E94A4
:101DB000C10E0C94C00E0E9489110E94E0030E9483
:101DC00027180C9465180E94891D0E9457120E94C2
:101DD000DB0E0E94C5150E94781A0C94C50E8F92D6
:101DE0009F92AF92BF92CF92DF92EF92FF920F93AA
:101DF0001F93CF93DF93CDB7DEB72A970FB6F89432
:101E0000DEBF0FBECDBF0E946C12982E81110E94C2
:101E10008F0E86E2A82E82E0B82E00E010E0802E21
:101E2000802F0E94AD11D82EF501C1905F01C82608
:101E3000B1F40F5F1F4F0330110589F78FEF8983CE
:101E40008A831B820E94921D8160782F9D838C83E0
:101E500049815A816B818D810E94FC032FC0809142
:101E6000350281FD0E94B311E12CFF24F3948C2DE7
:101E70008F21F1F00E94BE0E882399F0EE828F82AE
:101E8000DF2081E009F480E088870E94921D816054
:101E9000782F9A8789874E815F8168858A850E941D
:101EA000FC03F801EA5DFD4F8081F826F08206C050
:101EB000E394FF0CF3E0EF12DACFBBCF81E0911097
:101EC00001C080E02A960FB6F894DEBF0FBECDBFEA
:101ED000DF91CF911F910F91FF90EF90DF90CF9006
:101EE000BF90AF909F908F9008950E94EF0E0E9438
:101EF0008B170E948A1A81110E94A20E0E946614FA
:101F00000C94F103CF93DF930E94AF10EC01811585
:101F100021E5920708F045C0811530E5930708F0E8
:101F200094C0883E910528F5803E910508F0F8C0E0
:101F3000883A910570F4853A910508F07CC08130AB
:101F4000910509F475C008F4E8C0049708F0E8C0EA
:101F5000E4C08F3B910508F0E0C0C85AD0E0CC0F38
:101F6000DD1FC45BDE4F0990D881C02DCE01946483
:101F7000D8C0811540E2940758F4811551E09507C7
:101F800008F0CEC08D3E910508F4C7C09065C9C069
:101F9000C11580E4D80708F4C0C0DF70CE01906A94
:101FA000C0C0811525E59207A8F4811534E5930793
:101FB00008F095C0811543E5940708F07BC08115B2
:101FC00052E5950708F061C0D82FCC27CE01816F6C
:101FD000906AA7C0C11589E5D807A0F4C11528E506
:101FE000D20708F082C0C11536E5D30708F095C0C6
:101FF0008C2F0E9443118F7190E0D82FCC27CE01F7
:1020000090628FC0C1154AE5D40708F474C0CE01B0
:1020100090568115904208F080C08D2F8F710E94DC
:102020004311DD27D0628F71AE01582BCA0179C0F0
:1020300081E090E076C0C55AD0E0C658DE4F888176
:10204000C82FD0E0CE0190646CC074E0969587955F
:102050007A95E1F7282F23703C2F337081E090E0D0
:1020600002C0880F991F3A95E2F79C68AC01522B89
:102070009A019C2F9F709695969550E2959FE0014E
:102080001124C9018C2B9D2B4CC08370992721E012
:1020900030E002C0220F331F8A95E2F79C2F9695FD
:1020A000969580E2989FE0011124C22BD32BCE019C
:1020B0009C6837C08370992721E030E002C0220F6E
:1020C000331F8A95E2F79C2F9695969540E2949F50
:1020D000E0011124C22BD32BCE019A6822C0D82F45
:1020E000CC27CE01846F906A1CC0DC2FCC27CE0198
:1020F000806F906A16C08C2F8F700E94431194E0FD
:10210000D695C7959A95E1F7CF70D0E0DC2FCC2714
:10211000D0699E01282BC90104C080E090E001C075
:10212000CE01DF91CF910895272F30E0F901EE0F16
:10213000FF1F2E0F3F1FF90199E0899FE00DF11D50
:102140001124E60FF11DEE0FFF1FEA51FF4F85919D
:10215000949108950E9494100E94820F08958238ED
:10216000910569F1B0F48133910509F46DC048F42B
:102170008932910509F463C08A32910509F469C076
:1021800008958533910509F455C089339105B9F057
:102190000895833E910569F138F4803E9105B1F0D0
:1021A000823E910509F10895863E9105A9F1873E89
:1021B0009105B9F1843E910509F064C023C02091D6
:1021C0007D0220FD4FC021FD4DC0089580917D020C
:1021D00080FD44C080917E0280FF44C080917D02DA
:1021E00084FD42C083EE4DC080917D0282FF38C0E5
:1021F000F5CF80917D0282FD33C080917E0280FD0B
:1022000031C0ECCF80917E0281FF32C080917D028F
:1022100084FD2AC087EE35C080917D0283FF26C0F1
:10222000F5CF80917D0283FD21C080917E0281FDEA
:102230001FC0ECCF80917D0285FD1CC01DC0809128
:102240007D0285FD19C016C080917D0286FD16C0F5
:1022500017C080917D0286FD13C010C089E311C0B4
:1022600082EE0FC080EE0DC080E00BC086EE09C08C
:1022700084EE07C089E205C085E303C08AE201C09D
:1022800081E390E0089590917D0292FF0DC0282F88
:102290002871283019F4877F846006C0282F2471A4
:1022A000243011F48B7F886093FF0DC0282F287194
:1022B000283119F4877E846106C0282F24712431C7
:1022C00011F48B7E886120917E0220FF0DC0382F93
:1022D0003871383019F4877F816006C0382F31712A
:1022E000313011F48E7F886021FF0DC0282F2871B6
:1022F000283119F4877E816106C0282F2171213190
:1023000011F48E7E886194FD877E089580E00895A3
:1023100008950E94E00D811102C00E94880E0E9463
:10232000EB0D809335020E94F30D90937E02809313
:102330007D020E9488110E94EF0D682F70E080E0FE
:1023400090E00E94FF076091A2017091A30180912B
:10235000A4019091A5010C943708E82FF0E0EE5706
:10236000FD4F80810895089580EA8A95F1F70895D8
:1023700000C008950C94B41108950C94BC110C94F1
:10238000BD110C94BC110C94C111F894E82FE29586
:10239000EF70F0E031A1282F2F7081E090E001C0B4
:1023A000880F2A95EAF7982F9095932391A392A1ED
:1023B000892B82A37894089584E30E94C51185E354
:1023C0000E94C51186E30E94C51184E90E94C511CF
:1023D00086E90E94C51187E90C94C511EF92FF921E
:1023E0000F931F93CF93DF93C62FD0E0C358DE4FD8
:1023F00028812F3F09F454C0042F162F7C01F89434
:10240000E22FE295EF70F0E081A1422F4F7021E0C2
:1024100030E001C0220F4A95EAF7822B81A382A106
:102420002095282322A378940E94B81160E871E0D7
:10243000F701A7014D5F5F4FF12C302F3095DB0185
:102440002D91BD012F3FB1F0822F82958F7090E0CA
:10245000DC0190968C9190E02F7002C09595879545
:102460002A95E2F780FD06C08081802B8083FF24BF
:10247000F39403C08081832380833196E417F507AA
:10248000F1F688818F3F11F00E94C5116F2D812FC9
:10249000DF91CF911F910F91FF90EF900C94BA11A3
:1024A000DF91CF911F910F91FF90EF9008950E94BF
:1024B000DC1183E0E2E8F2E0DF01982F1D929A95AB
:1024C000E9F7EFE7F2E0DF011D928A95E9F783E093
:1024D0000E94AE120C94E8020F931F93CF93DF93E8
:1024E00000D01F92CDB7DEB719821A821B8210E08E
:1024F00001E0402F612FCE0101960E94EE111F5F77
:10250000000F1330B1F743E050E0BE016F5F7F4F23
:102510008FE792E00E945E2511E0009709F410E039
:10252000892B49F089819A81AB8180937F029093B6
:102530008002A0938102212F43E062E872E08FE7DE
:1025400092E00E94AF120E94EA02812F0F900F903A
:102550000F90DF91CF911F910F9108950895FF92F1
:102560000F931F93CF93DF938C01F62ED72FC42F99
:10257000222349F081E0809338020E94921D9093BB
:10258000370280933602809138028823C1F080910F
:102590003602909137020E94AA1D059780F0EF2D18
:1025A000FD2FD8014C2F50E0CD01801B910B8417DB
:1025B00095071CF48D918193F7CF10923802DF912B
:1025C000CF911F910F91FF9008950E94AA1F0E9422
:1025D000E30E0C94B61F0E94BA1F0E94750F0C9454
:1025E000D41F0E94301D0E94911F0E94CD0E0E9498
:1025F000E5120E94EB120E94D70EFBCF80913F02A2
:1026000080FF06C06091090170E0660F771F26C049
:1026100081FF04C06091090184E005C082FF07C00A
:102620006091090188E0689FB001112417C0909162
:102630003E029923D1F060910801961788F7209106
:10264000090188E0289F90011124929FA001939F87
:10265000500D112470E0CA010E94082560387105F0
:1026600040F46115710519F406C068E070E0862F2A
:1026700008958FE7089581E0089580913F0280FFDB
:1026800008C06091050170E075956795759567952F
:1026900021C081FF06C06091050170E075956795C6
:1026A00019C082FF04C06091050170E010C09091D4
:1026B0003D02992399F0609104019617A0F780914B
:1026C0000501899FC001112470E00E94082560382F
:1026D000710540F46115710519F406C061E070E000
:1026E000862F08958FE7089581E008958D3E21F4A7
:1026F0000E94FE12819504C08E3E29F40E94FE12B3
:102700008093430208958F3E21F40E94FE1281952A
:1027100004C0803F29F40E94FE1280934202089573
:10272000893F19F40E943D1305C08A3F31F40E948D
:102730003D1381958093440208958B3F21F40E94BC
:102740003D13819504C08C3F29F40E943D13809372
:10275000450208959FE0980F983078F421E030E02A
:10276000A90102C0440F551F9A95E2F7CA01909142
:102770004102892B8093410208958D3F21F480917D
:102780003F0281600BC08E3F21F480913F02826046
:1027900005C08F3F29F480913F02846080933F02FF
:1027A00008958D3E39F49091430297FF35C0109201
:1027B000430259C08E3E29F4909143021916BCF38E
:1027C0002BC0909142028F3E29F497FF25C01092B2
:1027D000420249C0803F19F41916CCF31DC09091F4
:1027E0004402893F29F41916BCF4109244023BC0FC
:1027F0008A3F19F497FF10C0F8CF8B3F39F49091BE
:10280000450297FF09C0109245022DC08C3F21F46C
:10281000909145021916BCF39FE0980F983080F410
:1028200021E030E0A90102C0440F551F9A95E2F75C
:10283000CA0180959091410289238093410213C07F
:102840008D3F21F480913F028E7F0BC08E3F21F49B
:1028500080913F028D7F05C08F3F29F480913F0218
:102860008B7F80933F0280914202811106C080914C
:102870004302811102C010923E02809144028111F4
:1028800006C080914502811102C010923D02089558
:102890000E94921D20914202211104C02091430206
:1028A000222321F090933C0280933B02209144022A
:1028B000211104C020914502222321F090933A0275
:1028C0008093390280E492E00C94FF1BEF92FF9218
:1028D0000F931F93CF93DF9300D000D000D0CDB7DC
:1028E000DEB786E0E0E4F2E0DE01119601900D92A1
:1028F0008A95E1F7E0904202F09043020091440291
:10290000109145021092420210924302109244022A
:1029100010924502E11003C0FF2009F45DC08091D0
:102920003B0290913C020E94AA1DAC0190913E0294
:10293000992339F020910A0130E02417350758F027
:102940004BC020910B018AE0289F9001112424178D
:10295000350718F041C09F3F19F09F5F90933E02EA
:10296000EE2061F00E94FE121E1414F09FEF01C0D1
:1029700091E0989F902D112490934202FF2061F0E6
:102980000E94FE121F1414F09FEF01C091E0989F67
:10299000902D112490934302309142023323E1F0B1
:1029A000209143022223C1F045EB3403C0011124DE
:1029B000992319F09093420203C081E08093420270
:1029C00035EB2303C0011124992319F0909343029E
:1029D00003C081E080934302011103C0112309F475
:1029E0005DC08091390290913A020E94AA1DAC010B
:1029F00090913D02992339F02091060130E024178F
:102A0000350758F04BC0209107018AE0289F9001BC
:102A100011242417350718F041C09F3F19F09F5F1C
:102A200090933D02002361F00E943D13101614F0B4
:102A30009FEF01C091E0989F902D11249093440244
:102A4000112361F00E943D13111614F09FEF01C095
:102A500091E0989F902D112490934502309144026B
:102A60003323E1F0209145022223C1F045EB3403EA
:102A7000C0011124992319F09093440203C081E00E
:102A80008093440235EB2303C0011124992319F0EC
:102A90009093450203C081E08093450280914202F9
:102AA00081110BC080914302811107C080914402C3
:102AB000811103C08091450281110E944814EB826C
:102AC000FC820D831E8386E0FE013196A0E4B2E015
:102AD00001900D928A95E1F726960FB6F894DEBF25
:102AE0000FBECDBFDF91CF911F910F91FF90EF905F
:102AF0000895E0E4F2E086E0DF011D928A95E9F7AF
:102B000010923E0210923D0210923F02089586E01C
:102B100090E00C946B25682F86E090E00C9479256A
:102B20008091850284708961809385020C948B1555
:102B30008091850286958695869508958091850277
:102B400081FD07C08260809385020E948B150C94E2
:102B50008C1708958091850281FF07C08D7F809337
:102B600085020E948B150C94981708958091850218
:102B700081FD0C94AA150C949E1580918502869572
:102B80008170089580910C0108950E94E00D8111DB
:102B900004C00E94880E0E9490150E9487158093A1
:102BA0008502282F26952695269530E0243031057C
:102BB00024F087708861809385028091850280FF70
:102BC00004C086958695869501C080E00C945917BF
:102BD00020918502822F869586958695482F50E014
:102BE0004330510554F48F5F982F990F990F990F27
:102BF000822F8770892B8093850280918502816066
:102C0000809385020E948B1580918502869586951A
:102C100086950C94591780918502982F96959695D4
:102C20009695A1F0915E990F990F990F8770892B56
:102C300080938502887F91E009F490E0809185027D
:102C400090FB80F9809385020E948B15809185020C
:102C50008695869586950C9459178091850280FDFE
:102C600013C0816080938502813019F489E08093DC
:102C70008502809185020E948B1580918502869540
:102C8000869586950C94591708958091850280FF4A
:102C900008C08E7F809385020E948B1580E00C9483
:102CA000591708958091850280FD0C9445160C9467
:102CB0002D1690918502892F8695869586958F5F32
:102CC0008F719770843038F4880F880F880F892BA4
:102CD0008093850202C09093850280918502887F4F
:102CE00091E009F490E08091850290FB80F9809357
:102CF00085020E948B158091850286958695869522
:102D00000C945917843008F083E0909185029770F5
:102D1000282F220F220F220F922B90938502987F4B
:102D200021E009F420E09091850220FB90F9909336
:102D300085020C9459170E948216809185020C948A
:102D40008B15FC01DB0112968C918823F9F0EC5B6A
:102D5000FC45E730F105D8F4EE59FF4F0C943E25C1
:102D600083E001C080E00E949B1680E008950E94ED
:102D70000B16FBCF0E94E815F8CF0E945216F5CF34
:102D80000E945916F2CF0E94B615EFCF81E0089548
:102D9000279A2F9808952F9808958F929F92AF9217
:102DA000BF92CF92DF92EF92FF920F931F93CF9338
:102DB000DF938C0180918600909187006CE070E039
:102DC0000E94F4246017710730F0C80169E070E0D8
:102DD0000E94F42460C08091860090918700E0906A
:102DE0008600F0908700E0918600F0918700C6E0B1
:102DF000D0E0BE010E94F42420E030E0060F171F4F
:102E0000211D311D4801590185E0880C991CAA1C1F
:102E1000BB1C8A95D1F7C701BE010E94F4246F0143
:102E2000E12CF12CA7019601260F371F411D511DE2
:102E3000C501B4010E941C2569017A01E091860058
:102E4000F0918700CA01B9010E94E4249B01AC0102
:102E5000DF010E9453259B01AC01C701B6010E940E
:102E6000E424DC01CB012FE0B695A79597958795D3
:102E70002A95D1F7009186001091870020E030E07C
:102E8000081719072A073B0728F4609186007091FC
:102E90008700CB01BC01CB01DF91CF911F910F9136
:102EA000FF90EF90DF90CF90BF90AF909F908F906A
:102EB0000895CF93C82F843050F4811109C08091B8
:102EC0008000877F809380000E94CB1606C0C3E0FD
:102ED00080918000886080938000A0918600B091EE
:102EE00087002C2F30E00E94442523E030E040E0B2
:102EF00050E00E941C25B42FA32F922F8827892FE2
:102F00009A2FAB2FBB270E94CD1690938D008093F4
:102F10008C00CF91089508951092470210924602B6
:102F200010924802EFE6F0E080818160808308958E
:102F3000EFE6F0E080818E7F80830E9498150C94EC
:102F400059171F920F920FB60F9211240F931F93D0
:102F50002F933F934F935F936F937F938F939F93A1
:102F6000AF93BF93CF93EF93FF9380910D0191E0C7
:102F7000980F823019F090930D0155C081E0809335
:102F80000D010E94C215C82F009146021091470200
:102F90000F5F1F4F0E94C21528E7829FB0011124C6
:102FA000C8010E94F424909347028093460228E7C8
:102FB000C29FB0011124660F672F661F770B7195B2
:102FC0000E94F4246F7780914802823019F46034B3
:102FD00051F404C0813039F46F3729F480916F00C7
:102FE0008E7F80936F00E62FF0E0E654FE4FC49191
:102FF00000918600109187000E949815282FC09F8D
:10300000C001C19F900D11246DEF72E00E94F42465
:10301000269FC001279F900D11240E94CD169093EA
:103020008D0080938C00FF91EF91CF91BF91AF9174
:103030009F918F917F916F915F914F913F912F91D0
:103040001F910F910F900FBE0F901F9018950E9427
:10305000C8168AE08093800089E1809381008FEF19
:103060009FEF90938700809386000E94C5150E9471
:10307000BD1581110C948C170895CF93DF9397FFA2
:103080000DC0FB012281222349F0EC010E947B1834
:10309000CE019F770E94EE180E94C81881E0DF9150
:1030A000CF91089590918702923069F48A3040F46C
:1030B00090E009966AE070E00E940825875A01C0F6
:1030C00086500C94ED040C94CF038CE090E00E94A9
:1030D0006B2590E0A0E0B0E0809387029093880297
:1030E000A0938902B0938A020895609187028CE0D0
:1030F00090E00C9479250E94E21B86958170809364
:103100008C020E94E21B817080938602809187026C
:10311000813039F480918C02882319F089E30E9470
:10312000ED040E94FA0C80938B020E940D0D809199
:103130008702813071F048F0823081F0843009F5E7
:1031400086EE0E94ED0488E11AC082EE0E944C04D3
:1031500018C088E193E00E94800213C0809186022B
:10316000811103C083E50E94ED0482EE0E944C04AD
:103170008FE39CE90197F1F700C0000087E50E940A
:10318000ED048FE39CE90197F1F700C0000008957A
:1031900080918702813059F030F0823089F084309C
:1031A000C9F488E215C082EE0E94A20413C08CE22A
:1031B0000E94ED0480918C02882361F089E308C0AD
:1031C00082EE0E94A20480918602811103C083E5F1
:1031D0000E94ED0480918B020C940A0D0F931F93B3
:1031E000CF93DF938C01CCE0D0E0C8010C2E02C05D
:1031F000969587950A94E2F78F700E94521824974B
:10320000CC3F8FEFD80789F7DF91CF911F910F91B6
:1032100008950F931F93CF93DF93EC018B01FB0174
:103220008281882361F00E94FA0CCE01825E9C4567
:103230008530910520F4809387020E947518B801AB
:10324000CE01DF91CF911F910F910C943D18CF9338
:10325000DF93EC01FB018281882309F43CC1C43077
:10326000FDE5DF0760F4CB3F9CE5D90788F49E01BC
:1032700022503C452431310508F02EC109C0C23628
:10328000EDE5DE0729F0C63AFDE5DF0709F024C1C8
:103290000E94F30D90937E0280937D02C1318CE5F4
:1032A000D80709F4C6C008F042C0C930ECE5DE0713
:1032B00009F49BC000F5C5308CE5D80709F485C03A
:1032C00078F4C330ECE5DE0709F478C008F07AC082
:1032D000C230DC4509F0F5C080917D028160EFC00D
:1032E000C7309CE5D90709F478C008F07AC080910E
:1032F0007D028061E4C0CD30FCE5DF0709F487C0C2
:1033000058F4CB309CE5D90709F479C008F07BC0AC
:1033100080917D0288606FC0CF30FCE5DF0709F443
:1033200080C008F082C080917D02877FC8C0CE3FF8
:103330009CE5D90709F471C000F5C531FCE5DF074C
:1033400009F485C068F4C3319CE5D90709F475C058
:1033500008F095C00E94A70780917D028F77AFC0CB
:10336000CC3FFCE5DF07A9F108F054C0CB3FDC45BA
:1033700009F0A7C080917E0240C0C230EDE5DE07B3
:1033800009F489C058F4C1158DE5D80709F45AC06D
:1033900008F069C080917E0282602FC0C236EDE5E0
:1033A000DE0709F47CC0C63AFDE5DF0709F481C0F9
:1033B000C330DD4509F085C080E06EC080917D029C
:1033C00082607DC080917D0216C080917D02886000
:1033D00076C080917E0282604FC080917D028062C3
:1033E0006EC080917D0280646AC00E94A7078091B0
:1033F0007D02806864C0846062C081603DC080914D
:103400007D028E7F5CC080917D028D7F58C080914F
:103410007D0216C080917E0218C080917E028D7F51
:103420002BC080917D028F7E4AC080917D028F7D6E
:1034300046C080917D028F7B42C080917D02877F54
:103440008B7F3DC080917E028D7F8E7F15C08091E5
:103450007D0282FB222720F991E0922790FB82F9DE
:1034600090FB83F92CC080917E02982F90959170EB
:103470008E7F892B90FB81F980937E0222C00E946F
:10348000A70780917D0287FB222720F991E09227F0
:1034900090FB87F914C081E00E948A0E12C08091CF
:1034A0007D0284FB222720F991E0922790FB84F98A
:1034B00006C080917D02982F909590FB80F98093B3
:1034C0007D0280917D0290917E020E94040E0E94F6
:1034D000A70780E001C081E0DF91CF9108958FE8D8
:1034E00091E00197F1F700C0000008950C941302D9
:1034F0005098589A5198599A0E946F1A89B1982FEA
:103500009170499902C080E001C082E0892B8093CC
:103510004B020895E0914B02EE0FEE0FE0934B0249
:1035200049B1842F817090E049B141FB222720F9F5
:1035300030E041FF02C022E030E0822B932B8E2B43
:1035400080934B028F70E82FF0E0ED57FE4F908193
:1035500080914A02890F80934A0284305CF0809106
:1035600049028F5F8093490260E080E00E94761AF2
:1035700021E001C020E080914A028D3F54F4809107
:10358000490281508093490261E080E00E94761AEE
:1035900021E080914A02082E000C990B64E070E053
:1035A0000E94082580934A02822F0895CF93DF93CB
:1035B00086319C4541F5EB010E94FA0C982F8A81D7
:1035C0002091020130910301882379F09A7A81E0F9
:1035D00009F480E080934C02911102C069E201C0BD
:1035E00065E3C9010E94CF1C0AC080914C02811181
:1035F00002C069E201C065E3C9010E94DA1C0E94B1
:103600003F0D80E001C081E0DF91CF9108950F93DD
:103610001F93CF93DF93C42FD22FFC018281882385
:10362000C9F040934F020E94921D90934E028093E6
:103630004D0280E28C0F883008F057C0C77081E0DF
:1036400001C0880FCA95EAF7DF91CF911F910F91C2
:103650000C94F60480914F02481330C080914D02C3
:1036600090914E020E94AA1D883C910538F510E207
:103670001D0FCD17B9F080E28C0F883040F4C77071
:1036800081E001C0880FCA95EAF70E94FD04183056
:1036900028F581E09D2F977001C0880F9A95EAF771
:1036A0000E94F604802F0E94ED041830F0F4D770C9
:1036B00081E001C0880FDA95EAF70AC080E28C0F3A
:1036C000883098F4C77081E001C0880FCA95EAF786
:1036D000DF91CF911F910F910C94FD04802FDF910A
:1036E000CF911F910F910C94ED04DF91CF911F9119
:1036F0000F9108950F939C01CB01243F4CE53407B3
:1037000031F188F4293DFCE53F07D9F02A3D4CE52D
:10371000340779F1283D3C45A9F506E221EE41EE5A
:1037200068ED7CE52BC0263FFCE53F07E1F0A8F003
:10373000273F3C4539F507E225EE46EE67EF7CE58D
:103740001DC007E225EE45EE69ED7CE517C006E2F7
:1037500021EE40EE64EF7CE511C007E225EE44EE79
:1037600065EF7CE50BC006E221EE42EE66EF7CE5FC
:1037700005C008E221E045EE6AED7CE50E94071BEA
:1037800080E008C0FC018281882319F010924F026A
:1037900001C081E00F910895909395018093940169
:1037A000089590935502809354020895E091540235
:1037B000F0915502309721F00190F081E02D0994AD
:1037C00080E008950E94D61B0895E0915402F09184
:1037D0005502309799F020911A01222359F0209137
:1037E0007D0227FF07C0DC012C9111962C931197C5
:1037F00026E02C930280F381E02D09940895E09156
:103800005402F0915502309739F022E0DC012C93FC
:103810000480F581E02D09940895209152023091A1
:1038200053022817390771F0909353028093520284
:10383000E0915402F0915502309721F00680F78113
:10384000E02D0994089520915002309151022817DB
:10385000390771F09093510280935002E091540225
:10386000F0915502309721F00084F185E02D099404
:103870000895FC01329680911A01882331F08091DD
:103880007D0287FF02C09EE101C096E080E091507A
:1038900028F021912223D9F38F5FF9CF0895662371
:1038A00051F120911A012223E9F020917D0227FF96
:1038B00019C0462F4695469546954E31E0F46770FF
:1038C00021E030E002C0220F331F6A95E2F7FC01CD
:1038D000E40FF11D828190E02823392381E0232B1E
:1038E00069F409C0FC01329608962191621729F00B
:1038F000E817F907D1F780E0089581E008959C0169
:10390000FC0132969FEF80E04191461789F09F3F7E
:1039100019F4411101C0982F8F5F8630A9F79F3F9E
:1039200039F0F901E90FF11D97FDFA9562830895C9
:1039300008959C012A5F3F4FFC014281461301C05C
:103940001282019682179307B9F70895262F2695BC
:10395000269526952E3168F4FC01E20FF11D677063
:1039600021E030E001C0220F6A95EAF78281282B1E
:1039700022830895262F2695269526952E3170F4BC
:10398000FC01E20FF11D677021E030E001C0220F61
:103990006A95EAF720958281282322830895209151
:1039A0001A01222329F020917D0227FD0C94A61CE8
:1039B0000C947F1C20911A01222329F020917D0272
:1039C00027FD0C94BA1C0C94991C20911A01FC013F
:1039D0003296222331F080917D0287FF02C08EE172
:1039E00001C086E0DF011D928A95E9F708950895E8
:1039F0000C94F71C83E0809356020C94F81C811100
:103A000002C081E001C082E0809356020C94F81C51
:103A10000C94FF1C81E0809356020C94F81C0C94CB
:103A20000A1D08950C94111D0C94121D0C94111D67
:103A30000C94111D0C94111DCF930E94181D0E940F
:103A40006C120E94161DC0E08C2F0E94AD118111D6
:103A500004C0CF5FC330C1F701C081E0CF910895AA
:103A600008951F920F920FB60F9211248F939F9378
:103A7000AF93BF9380915702811113C080918D0243
:103A800090918E02A0918F02B09190024196A11D5B
:103A9000B11D80938D0290938E02A0938F02B093FC
:103AA0009002BF91AF919F918F910F900FBE0F9099
:103AB0001F90189580919502843031F10E945C032B
:103AC0001092570220E488E190E00FB6F894A89590
:103AD000809360000FBE2093600083B7817F846075
:103AE00083BF83B7816083BF7894889583B78E7FC7
:103AF00083BF0FB6F894A895809160008861809389
:103B00006000109260000FBE08950E94A7070C94F9
:103B1000630382E084BD93E095BD9AEF97BD8093E7
:103B20006E0008952FB7F89480918D0290918E02C7
:103B3000A0918F02B09190022FBF08952FB7F894F3
:103B400060918D0270918E0280918F02909190020F
:103B50002FBF08959C014FB7F89480918D029091EA
:103B60008E02A0918F02B09190024FBF821B930BE7
:103B7000089578941F920F920FB60F9211248F938D
:103B80009F93AF93BF9380918D0290918E02A091ED
:103B90008F02B09190020196A11DB11D80938D02FC
:103BA00090938E02A0938F02B0939002BF91AF9139
:103BB0009F918F910F900FBE0F901F90189581E0ED
:103BC0008093E00080E28093D8001092C9008FE1DA
:103BD0009EE40197F1F700C0000087E090EBDC0164
:103BE00080939E0290939F02A093A002B093A102A3
:103BF0009CE088E10FB6F894A895809360000FBE12
:103C000090936000FFCF80917B020895089522E099
:103C10002093E9002FEF3091E800215035FD06C0D8
:103C200035ED3A95F1F700002111F5CF2091E8002C
:103C300025FF0BC040E050E066E070E00E944620A7
:103C40008091E8008E778093E8000895CF93DF930A
:103C500020911A01222339F020917D0227FF03C011
:103C600060E222E002C068E021E02093E9002FEF4B
:103C70003091E800215035FD06C035ED3A95F1F759
:103C800000002111F5CF2091E80025FF1DC0EC01B7
:103C900080911A01811105C040E050E068E070E0B9
:103CA00003C070E040E050E0CE010E9446208091C9
:103CB000E8008E778093E80080E2FE01ABE5B2E099
:103CC00001900D928A95E1F7DF91CF91089580934D
:103CD000580270935A026093590280919502843081
:103CE00001F582E08093E9008FEF9091E800815028
:103CF00095FD06C095ED9A95F1F700008111F5CF7D
:103D00008091E80085FF0DC040E050E063E070E086
:103D100088E592E00E9446208091E8008E778093AB
:103D2000E8000895BC0184E00C94671EBC0183E0A8
:103D30000C94671E80919402811109C00E94D721C2
:103D40000E9434228091E20084608093E200089512
:103D50001092940208950C940F1D6091910281E0DD
:103D6000611101C080E00C94FA1C9091950281E0F1
:103D7000943009F080E0609191020C94FF1C42E0C5
:103D800061EC81E00E94502142E261EC82E00E94FD
:103D900050219091950281E0943009F080E060918B
:103DA00091020C94081D80919702833009F461C040
:103DB00030F4813071F0823009F49AC008958A306D
:103DC00009F486C08B3009F46CC0893009F0A8C0B2
:103DD00020C080919602813A09F0A2C08091E8004B
:103DE000877F8093E80080919A0290919B02892BB3
:103DF00021F460E28BE592E003C060E080E090E0B7
:103E000070E00E9491208091E8008B778093E80019
:103E1000089580919602813209F082C080919A02C1
:103E200090919B02029708F07BC08091E800877F09
:103E30008093E8008091E80082FD05C080919502A2
:103E40008111F8CF6DC02091F3008091F20090E0D5
:103E5000922B029731F48091F100813011F086307D
:103E600021F48091F10080937B028091E8008B77B0
:103E700053C080919602813A09F052C080919A0213
:103E800090919B02892B09F04BC08091E800877FBD
:103E90008093E8008091E80080FFFCCF80911A01B8
:103EA00036C0809196028132D9F580919A02909124
:103EB0009B02892BA9F58091E800877F8093E80019
:103EC0000E9485218091980280931A010C94A70783
:103ED00080919602813221F58091E800877F80935E
:103EE000E8000E9485218091990280937C020895C8
:103EF00080919602813AA1F48091E800877F8093B7
:103F0000E8008091E80080FFFCCF80917C028093E4
:103F1000F1008091E8008E778093E8000C94852171
:103F2000089584B7877F84BF0FB6F894A8958091D1
:103F30006000886180936000109260000FBE90E086
:103F400080E80FB6F89480936100909361000FBEF3
:103F50000C940A1D0E94D7210E943422E2EEF0E068
:103F600080818460808378940C94C9248EE091E0F1
:103F70000C94D11B809195028530A9F48091950213
:103F8000853079F40E945A1D809193028823B1F301
:103F90000E941C1D882391F30E9430200E94A707D5
:103FA000EDCF0C94851D089508950C94D71F292FEB
:103FB000332723303105C9F060F42130310581F019
:103FC0002230310509F044C08BE390E02EE632E068
:103FD00043C021323105E1F02232310549F138C0C8
:103FE00082E190E029EA32E037C0992781309105DB
:103FF00049F028F0029761F5EAE3F2E005C0EAE64D
:10400000F2E002C0E0E5F2E0849190E09F0124C07C
:104010006115710541F061307105D1F489E090E0DE
:1040200029E932E019C089E090E020E832E014C0CC
:104030006115710541F06130710551F486EB90E036
:104040002BEB32E009C080E490E021E733E004C0CC
:1040500080E090E020E030E0FA0131832083089591
:1040600080E189BD82E189BD09B400FEFDCF809168
:10407000D8008F7D8093D8008091E000826080938B
:10408000E0008091E00081FDFCCF0895CF92DF92A7
:10409000EF92FF920F931F93CF93DF93EC018B016D
:1040A0007A010E94A421811133C0E114F10439F096
:1040B000F70180819181081B190BC80FD91FC12CF2
:1040C000D12C0115110519F18091E80085FD16C06C
:1040D0008091E8008E778093E800E114F10449F0C4
:1040E000F70180819181C80ED91ED182C08285E0FE
:1040F0000FC00E94A421882321F30AC089918093D4
:10410000F10001501109FFEFCF1ADF0ADACF80E08A
:10411000DF91CF911F910F91FF90EF90DF90CF90A3
:10412000089520919C0230919D022617370748F090
:104130006115710539F42091E8002E772093E8008D
:1041400001C0B901FC0120E06115710579F1809190
:1041500095028823F1F18530F1F18091E80083FD2B
:104160003CC08091E80082FD2EC08091E80080FF75
:10417000EBCF2091F3008091F20090E0922B61153B
:10418000710551F08830910538F421912093F100A8
:10419000615071090196F3CF21E0089709F020E002
:1041A0008091E8008E778093E800CECF2111CFCFA9
:1041B0000AC080919502882361F0853061F080917A
:1041C000E80083FD0AC08091E80082FFF2CF80E022
:1041D000089582E0089583E0089581E00895209194
:1041E0009C0230919D022617370748F06115710532
:1041F00039F42091E8002E772093E80001C0B9013E
:10420000FC0120E06115710591F1809195028823F0
:1042100009F440C0853009F43FC08091E80083FD77
:104220003DC08091E80082FD2FC08091E80080FFB2
:10423000E9CF2091F3008091F20090E0922B61157C
:10424000710559F08830910540F424912093F100D4
:104250003196615071090196F2CF21E0089709F07B
:1042600020E08091E8008E778093E800CBCF211189
:10427000CCCF0AC080919502882361F0853061F02F
:104280008091E80083FD0AC08091E80082FFF2CFB0
:1042900080E0089582E0089583E0089581E0089524
:1042A000982F973068F59093E900981739F070913E
:1042B000EC002091ED005091F00003C0242F762FE8
:1042C00050E021FD02C09F5FECCF3091EB003E7FBC
:1042D0003093EB003091ED003D7F3093ED00309155
:1042E000EB0031603093EB007093EC002093ED0015
:1042F0005093F0002091EE0027FDE5CF80E0089577
:104300008F708093E90081E008958091960287FF85
:1043100011C08091E80082FD05C080919502811155
:10432000F8CF11C08091E8008B770BC08091950287
:10433000882349F08091E80080FFF8CF8091E80061
:104340008E778093E80008952091E4003091E50095
:1043500095E64091EC00842F817040FF23C080914E
:10436000E80080FD1DC080919502882399F085307A
:1043700099F08091EB0085FD11C04091E4005091CF
:10438000E5002417350729F3915011F09A01E1CF88
:1043900084E0089582E0089583E0089581E008951F
:1043A00080E008954091E80042FFDDCF08950E942B
:1043B00045220E944D22E0EEF0E080818160808302
:1043C000E8EDF0E080818F77808319BCA7EDB0E045
:1043D0008C918E7F8C9380818F7E8083109294024B
:1043E00008950F931F93CF93DF930E9445220E945D
:1043F0004D22C8EDD0E088818F77888388818068DE
:10440000888388818F7D888319BC109295021092D1
:104410009102109293021092920200EE10E0F801C5
:1044200080818B7F808388818160888342E060E027
:1044300080E00E945021E1EEF0E080818E7F808359
:10444000E2EEF0E0808181608083808188608083FB
:10445000F80180818E7F8083888180618883DF91ED
:10446000CF911F910F910895E8EDF0E080818F7E4C
:104470008083E7EDF0E080818160808384E082BF0B
:1044800081E0809394020C94F121E8EDF0E08081CA
:104490008E7F80831092E20008951092DA001092CD
:1044A000E10008951F920F920FB60F9211242F93DF
:1044B0003F934F935F936F937F938F939F93AF93AC
:1044C000BF93EF93FF938091E10082FF0BC0809137
:1044D000E20082FF07C08091E1008B7F8093E100C2
:1044E0000E94C8248091DA0080FF1FC08091D8000C
:1044F00080FF1BC08091DA008E7F8093DA0080916C
:10450000D90080FF0DC080E189BD82E189BD09B479
:1045100000FEFDCF81E0809395020E949A1E05C0A7
:1045200019BC109295020E94A81E8091E10080FFA4
:1045300019C08091E20080FF15C08091E2008E7F5B
:104540008093E2008091E20080618093E20080919C
:10455000D80080628093D80019BC85E080939502D2
:104560000E94AD1E8091E10084FF30C08091E20086
:1045700084FF2CC080E189BD82E189BD09B400FEC1
:10458000FDCF8091D8008F7D8093D8008091E1008D
:104590008F7E8093E1008091E2008F7E8093E20025
:1045A0008091E20081608093E200809191028823F3
:1045B00011F084E007C08091E30087FD02C081E034
:1045C00001C083E0809395020E94B51E8091E100B6
:1045D00083FF29C08091E20083FF25C08091E10024
:1045E000877F8093E10082E0809395021092910290
:1045F0008091E1008E7F8093E1008091E2008E7FC8
:104600008093E2008091E20080618093E20042E0CA
:1046100060E080E00E9450218091F00088608093EB
:10462000F0000E94AB1EFF91EF91BF91AF919F915F
:104630008F917F916F915F914F913F912F910F904B
:104640000FBE0F901F9018951F920F920FB60F92EA
:1046500011242F933F934F935F936F937F938F9387
:104660009F93AF93BF93CF93DF93EF93FF93C0914B
:10467000E900CF708091EC00D82FD17080FDD0E898
:104680001092E9008091F000877F8093F000789489
:104690000E9468231092E9008091F0008860809366
:1046A000F000CD2BCF70C093E900FF91EF91DF9127
:1046B000CF91BF91AF919F918F917F916F915F91BA
:1046C0004F913F912F910F900FBE0F901F90189513
:1046D0001F93CF93DF93CDB7DEB7AA970FB6F894A9
:1046E000DEBF0FBECDBFE6E9F2E08091F10081931D
:1046F00022E0EE39F207C9F70E94D31E8091E8004C
:1047000083FF2EC18091960290919702492F50E02D
:104710004A30510508F024C1FA01E759FF4F0C94C3
:104720003E25803821F0823809F01AC108C08091F6
:10473000920290919302992389F082600FC0809138
:104740009A028F70873008F00BC18093E900809146
:10475000EB0085FB882780F91092E9009091E80032
:10476000977F9093E8008093F1001092F100D1C000
:10477000282F2D7F09F0F4C0882319F0823061F0D2
:10478000EFC080919802813009F0EAC0933009F0BF
:1047900080E0809393022EC08091980281112AC0FC
:1047A00080919A028F702FEF280F263008F0D8C022
:1047B0008093E9002091EB0020FF1CC0933021F48E
:1047C0008091EB00806214C09091EB009061909317
:1047D000EB0021E030E0A90102C0440F551F8A958B
:1047E000E2F74093EA001092EA008091EB008860C3
:1047F0008093EB001092E9008091E800877F80931E
:10480000E8000E948521ACC08111AAC010919802D5
:104810001F778091E3008078812B8093E300809163
:10482000E800877F8093E8000E9485218091E8005E
:1048300080FFFCCF8091E30080688093E30011113A
:1048400002C082E001C083E08093950289C0805855
:10485000823008F085C080919802909199028C3D39
:1048600053E0950779F583E08A838AE289834FB71D
:10487000F894DE01139620E03EE051E2E32FF0E0F1
:1048800050935700E49120FF03C0E295EF703F5F23
:10489000EF708E2F90E0EA3010F0C79601C0C096FE
:1048A0008D939D932F5F243149F74FBF8091E8008E
:1048B000877F8093E8006AE270E0CE0101960E9453
:1048C000912016C060919A0270919B02AE014F5FD9
:1048D0005F4F0E94D51FBC01892B09F441C0909104
:1048E000E800977F9093E80089819A810E94EF20E9
:1048F0008091E8008B778093E80032C0803881F5A2
:104900008091E800877F8093E800809191028093F6
:10491000F1008091E8008E7772CF811121C08091E3
:1049200098029091990299270297D4F48091E80017
:10493000877F8093E80080919802809391020E9483
:10494000852180919102811106C08091E30087FD4D
:1049500002C081E001C084E0809395020E94BF1EE6
:104960008091E80083FF0AC08091E800877F8093F0
:10497000E8008091EB0080628093EB00AA960FB66E
:10498000F894DEBF0FBECDBFDF91CF911F91089588
:104990000895CF93809195028823A1F0C091E900FA
:1049A000CF709091EC00892F817090FD80E8C82B2A
:1049B0001092E9008091E80083FD0E946823CF7087
:1049C000C093E900CF910895DB018F939F930E94DC
:1049D0005325BF91AF91A29F800D911DA39F900D74
:1049E000B29F900D11240895AA1BBB1B51E107C073
:1049F000AA1FBB1FA617B70710F0A61BB70B881F6F
:104A0000991F5A95A9F780959095BC01CD010895FD
:104A100097FB072E16F4009407D077FD09D00E946B
:104A2000F42407FC05D03EF4909581959F4F08959E
:104A3000709561957F4F0895A1E21A2EAA1BBB1BAA
:104A4000FD010DC0AA1FBB1FEE1FFF1FA217B3075A
:104A5000E407F50720F0A21BB30BE40BF50B661F70
:104A6000771F881F991F1A9469F760957095809534
:104A700090959B01AC01BD01CF010895EE0FFF1F82
:104A80000590F491E02D0994A29FB001B39FC0015D
:104A9000A39F700D811D1124911DB29F700D811D6A
:104AA0001124911D08950E944425A59F900DB49F47
:104AB000900DA49F800D911D11240895FB01DC0130
:104AC00004C08D910190801921F441505040C8F7E5
:104AD000881B990B0895F999FECF92BD81BDF89A74
:104AE000992780B50895A8E1B0E042E050E00C9429
:104AF0009F25262FF999FECF92BD81BDF89A019787
:104B000000B4021639F01FBA20BD0FB6F894FA9A15
:104B1000F99A0FBE08950396272F0E947A250E94C6
:104B20007925252F0E947A25242F0C947A25019629
:104B3000272F0E947A250C947925DC01CB01FC01FA
:104B4000F999FECF06C0F2BDE1BDF89A319600B4E6
:0E4B50000D9241505040B8F70895F894FFCFF1
:104B5E00C8000402280850011E0A14010601031E93
:104B6E00261E071E961E921E061E01E200E900EA90
:104B7E0000B500B600B700CD008301CC008A0192CB
:104B8E000194012102230224022502260227022A71
:104B9E0002B300B4006F007000818283E200E9006E
:104BAE00EA00B500B600B700CD008301CC008A0143
:104BBE0092019401210223022402250226022702D9
:104BCE002A02B300B4006F00700081828334353640
:104BDE0094969700FF0100010000FFFF0000010006
:044BEE0001FF0000C3
:00000001FF
